:020000040000FA
:0400000000002E28A6
:080008008B138C1C20288C10C6
:100010005C1C1528861656088E0057088F000C1099
:10002000101483160C1483122C28061650088E0008
:1000300051088F000C10101483160C1483122C28F6
:100040000C1C2C280C1010105C1C292886125C102B
:100050002C2806125C142C288B170900F130D700CD
:10006000D100F030D600D000F530DB007430DA007B
:10007000EE30D9006C30D800F530D5007430D400A3
:10008000EE30D3006C30D2002130A0000030C3002D
:10009000A100A200A300A400A500A600A700A8003C
:1000A000DE013A30B8008312B901380884003908FB
:1000B000840783169B001C141A0883128000B90A57
:1000C00005303902031D55285A30B200B300B40080
:1000D0003930B500B6003230B000B1013A30B80066
:1000E000B901C001C101C3018316CF30860083125C
:1000F00083167430920083127F30920083164D3045
:100100009900203098008312903098008B170B17BD
:1001100083168C1483128B178C1E8C288B131A0851
:10012000C2008C1299004118C528C01BBE28300897
:1001300084003108840700084202031DA928B10A7F
:1001400005303102031DAA28B101B901FF30C000FA
:100150008B28B1013808840039088407000842025E
:10016000031DBC28B90A05303902031D8B28B101D3
:10017000B901FF30C0008B28B9018B284208031950
:100180002E28C000FF30C1008B280613013040022A
:100190000319D128023040020319E828C001C10127
:1001A0008B28200884004308840742088000C30A83
:1001B00006304302031D8B28C301C001C101210881
:1001C000D0002208D1002308D6002408D7008B28AD
:1001D000380884003908840742088000B90A0530CD
:1001E0003902031D8B28B901C001C1013808840000
:1001F00039088407000883169A0083123908831689
:100200009B009C111C1555309D00AA309D009C142C
:100210001C1183128C1F0A298C13B90A053039026C
:0C022000031DF628B901C001C1018B28A4
:02400E00613F10
:10420000560047005900390039002000530045008E
:10421000520056004F002000560030002E003000A3
:00000001FF
